:100000000C943E040C94AA040C941A080C94AA04B0
:100010000C94C6090C94AA040C94AA040C94AA0487
:100020000C94AA040C94AA040C945E1F0C94AA04C9
:100030000C94D92D0C94AA040C94AA040C94AA0430
:100040000C94AA040C94AA040C94AA040C94AA0478
:100050000C94AA040C942E2E0C94AA040C94AA04BA
:100060000C94AA040C94AA040C94AA040C94AA0458
:100070000C94AA040C94AA040C94AA040C94AA0448
:100080000C94AA040C94AA040C94AA040C94AA0438
:100090000C94AA040C94AA040C94AA040C94AA0428
:1000A0000C94AA040C94AA040C94AA04460D540DB2
:1000B000600D600D380D600D600D600D600D600D00
:1000C000600D600D600D600D600D600D600D600DC8
:1000D0003A0D600D3C0D600D600D600D600D580D0A
:1000E000600D6F0D560D600D600D600D600D600DA3
:1000F000600D600D600D600D600D600D600D600D98
:10010000300D4C0D3E0D500D600D400D600D440D39
:10011000600D4E0D420D520D480D4A0D600D600DE3
:10012000600D600D600D600D600D320D340D360DEB
:100130005A0D5C0D600D600D600D5E0D0C0E0E0E07
:10014000180E180E180E180E180E180E100E120E8D
:10015000D40D180E180E0E0E1B0E180E180ED40D00
:100160000C0E180E180E120E180E180E180E180E71
:10017000180E180ED60D0C0EF80D180EFC0D180EDC
:10018000180E180ED80D100E180E180E060E180E9A
:10019000180E180EDA0D160E180EFA0D180E0E0E99
:1001A000180E180E0A0EFE0D180E000E120E180E66
:1001B000180E180E080E020E180E180E180E180E35
:1001C000180E180E180E040E180EDC0D180E180E50
:1001D000100E180E180E160E180E180E180E180EF9
:1001E000180E180E180E180E180EDE0D180E180E1A
:1001F000180E060E180E180E180E180E180E180EE1
:10020000180E180E180E180EE00D180EE20DE40D63
:10021000180E180E180EE60DE80DEA0D180EEC0D6E
:10022000EE0D180E180E180E140EF00D180EF40D1B
:10023000F20DF60D180E180E180E180E160EBA0E38
:10024000080FE70E2E0F520F5A0F610F660F6A0F3D
:10025000710F7E0F9D109F10A110A310A510AD105F
:10026000AD10AD10A710A910AB1081119911AD11EF
:10027000C811DA11E5110912221248126A124F133D
:10028000F414F116D616AC1DD31DCB1ED31DCB1EF8
:100290001F1E421ECB1E991EA81EC623C623FE2368
:1002A000FE237924AD24A426A426C424A426552400
:1002B00055245E26A42673269126722530325820B6
:1002C000005220006973723A253034582000772597
:1002D0003032582000214353335F4630210A002139
:1002E0004353335F5245414459210A00214353335C
:1002F0005F5245534554210A00214353325F453034
:100300005F4630210A00214353325F4630212025C9
:100310003032580A00214353325F4530210A002110
:100320004353325F494E4954210A00214353315F00
:1003300045305F25303258210A0045257520005090
:10034000257520004D5B783A256420793A25642094
:10035000763A256420683A256420623A253032587E
:100360005D0A000A5B434C525D20004C257520005D
:100370000A4D6F7573653A2025730A000A44454695
:100380003A20000A4558503A20000A494E543A2073
:10039000000A4C4F473A20000A4C4D533A20005374
:1003A000257520000A49443A2530345828257325FC
:1003B000732920000A556E6B6E6F776E2049443AA0
:1003C000205265706F727420746F20544D4B200062
:1003D0004E4720004F4B20004E4720004F4B20003F
:1003E0000A353537365F43533832683A005225753F
:1003F00020005725752000572575200057257520AA
:1004000000582575200041257520004925752000DC
:100410005B4348475D20000A2575205052543A2519
:10042000303258204953523A2530345820000A259A
:1004300075204552523A25303258204953523A25B8
:100440003034582000535B25303258202530325844
:1004500020253032585D2000007B46010203763AA9
:10046000687F6577482B353B6978796439141E3C81
:100470006A7A1D16041A1F3D6B061B070821203ED1
:100480006C2C19091715223F6D11050B0A1C23400E
:100490006E7E100D182425416F360E0C1227264251
:1004A0007037380F33132D43717534322F2E447249
:1004B0007C7D28303174457351504A524D492A543D
:1004C00066594F5C5F4C4B4E62635A5D5E602953C8
:1004D00067585B56576147554842403E3C3A3B455A
:1004E0006843413F3D2B357E697A790078141E7B45
:1004F0006A7C1D16041A1F7F6B061B0708212065E6
:100500006C2C19091715224A6D11050B0A1C234C76
:100510006E49100D182425516F360E0C1227264FE8
:100520007037380F33132D52717534502F2E4E7291
:10053000397D28304D314B735464586776012A77E2
:100540003259745C5F66020362635A5D5E602953D0
:1005500044575B565561474680291E1F20212223A0
:10056000242526272D2E2A2B141A0815171C180CA3
:1005700012132F302878041607090A0B0D0E0F33BB
:10058000343579311D1B06190511103637387D5564
:100590007A2C393A3B3C3D3E3F4041424353475F12
:1005A0006061565C5D5E57595A5B626346486444BD
:1005B00045677B7F650301025250514F68696A6B42
:1005C0006C6D6E6F7071725800494C754A4D734B6B
:1005D0004E767C777E7466540A4C6F6F702073740D
:1005E0006172742E0A000A55534220636F6E666969
:1005F00067757265642E0A000A544D4B3A633230B7
:100600003561352F4C5546413A6436613764660A88
:10061000003403490042004D0020005000430020F8
:10062000006B006500790062006F00610072006479
:1006300000200063006F006E007600650072007499
:1006400000650072000000080354004D004B0000DC
:10065000000403090409025400030100A032090444
:1006600000000103010100092111010001223900EC
:1006700007058103200001090401000103010200B4
:10068000092111010001227F0007058203080001F2
:1006900009040200010300000009211101000122E8
:1006A0002200070583032000011201100100000051
:1006B00008EDFEEE1B0102010200010631FF097484
:1006C000A1010975150026FF009520750881020912
:1006D00076150026FF00952075089102C0050109D6
:1006E00002A1010901A100850105091901290815C7
:1006F00000250195087501810205010930093115B0
:1007000081257F95027508810609381581257F9519
:100710000175088106050C0A38021581257F9501AF
:1007200075088106C0C005010980A1018502160176
:10073000002637001A81002AB70075109501810044
:10074000C0050C0901A1018503160100269C021AAF
:1007500001002A9C02751095018100C0050109065F
:10076000A101050719E029E7150025019508750184
:100770008102050819012905950575019102950168
:10078000750391010507190029F71500250195F852
:1007900075018102C0636F6E73756D65723A2025B5
:1007A0003034580A0073797374656D3A20253034FB
:1007B000580A000A002530325820006B6579626FB4
:1007C0006172643A20004C45443A20253032580A80
:1007D0000025583A253031366225730A000A202058
:1007E0003031323334353637383941424344454667
:1007F0000A0064656C5F6B65795F6269743A2063B7
:10080000616E27742064656C3A20253032580A00E6
:100810006164645F6B65795F6269743A2063616EDD
:100820002774206164643A20253032580A00290A6E
:10083000002575002F002575005D28002564002027
:1008400000256400200025640020002564007C0051
:1008500025303258006D6F7573656B6579205B626A
:10086000746E7C782079207620685D287265702F00
:1008700061636C293A205B00720B801711241FBE44
:10088000CFEFDAE0DEBFCDBF04B603FE41C08091FA
:10089000220490912304A0912404B0912504873070
:1008A000904BA740B04BA1F5109222041092230464
:1008B000109224041092250414BE0FB6F894A89543
:1008C00080916000886180936000109260000FBE8C
:1008D0001092010810920008E3E0F0E089E08093B4
:1008E0005700E491E695E370E150E33040F4F0E026
:1008F000EE0FFF1FE858FE4F8081918102C080E01B
:1009000090E1E0E0F0E8E81BF90BF695E795099532
:1009100011E0A0E0B1E0E0E1F5E602C005900D9243
:10092000AE37B107D9F724E0AEE7B1E001C01D92C0
:10093000A232B207E1F714E0CEE3D4E004C021977D
:10094000FE010E946C32CC33D107C9F70E94BF1A56
:100950000C9486320C940000FF93EF93E0917E019B
:10096000F0917F01309709F00995EF91FF9108957B
:10097000FC018591803011F0EFDFFBCF0895FF2758
:10098000E0E230E247FF0CC0419597FF09C0EDE27D
:100990006095709580959095611D711D811D911DCB
:1009A00027FF02C0219530E350E2AA27660F771F88
:1009B000881F991FAA1FA41710F0A41B63955A95AE
:1009C000A9F7AA3008F0A95FA05DAF93F395611570
:1009D00071058105910541F7ED3211F4EF93F3951F
:1009E000F21718F43F93F395FBCF8F91B5DFFA958B
:1009F000E1F70895E991F9918591803021F08532F0
:100A000019F0AADFF9CF089520E0E8945591553206
:100A1000C1F3503311F4689455915A3348F450534C
:100A200090F3220F022E220F220F200D250FF4CF5C
:100A30000EF4219589919991533619F3533729F181
:100A4000533559F1BC0188279927E8945C3621F485
:100A50008991999168945591543639F446EF7EF016
:100A600077FF0DC08FEF9FEF0AC055374AE039F08E
:100A7000583540E121F0523642E009F00895FF93E5
:100A8000EF937DDFEF91FF91B7CFFF93EF93FC01E1
:100A900081918030B9F360DFFBCFFF93EF9368DF84
:100AA000F1CFDF93CF93CDB7DEB72596A3DFCF91FC
:100AB000DF910895FC012AB1938D909592239AB904
:100AC0009BB1838D892B8BB90895FC019AB1838DDD
:100AD000809589238AB99BB1838D892B8BB985E059
:100AE0008A95F1F7000099B1838D982381E009F48C
:100AF00080E00895FC012BB1948D909592239BB9D1
:100B00009AB1848D892B8AB90895FC012AB1948DFC
:100B1000909592239AB99BB1848D892B8BB90895B6
:100B2000FC019AB1848D809589238AB99BB1848D0B
:100B3000892B8BB985E08A95F1F7000099B1848DF6
:100B4000982381E009F480E008950F931F93CF93D9
:100B5000DF938C01EB01C8010E946505882341F0F9
:100B6000209731F085E08A95F1F700002197F3CFC7
:100B7000CE01DF91CF911F910F9108950F931F9395
:100B8000CF93DF938C01EB01C8010E9465058111B1
:100B900008C0209731F085E08A95F1F70000219791
:100BA000F3CFCE01DF91CF911F910F910895CF9395
:100BB000DF93EC010E945A05CE01DF91CF910C9496
:100BC00085053BB1FC01238D209523232BB93AB138
:100BD000238D232B2AB90C948505FC018CB3938DAE
:100BE000982B9CBB9DB3838D892B8DBB0895CF9390
:100BF000DF93EC010E94ED05CE01DF91CF910C94C3
:100C0000D705FC012DB3938D909592239DBBCF0109
:100C10000C94E105FC01118210821282138280E0A3
:100C200090E895838483178210860895CF93DF938D
:100C3000EC012E9826982F9827980E94E105898D1F
:100C4000843080F440916900880F22E030E0B901DF
:100C500002C0660F771F8A95E2F7CB01842B809341
:100C6000690010C040916A008370880F22E030E074
:100C7000B90102C0660F771F8A95E2F7CB01842B7A
:100C800080936A009DB38B8D809589238DBBCE01A7
:100C9000DF91CF910C940A06CF93DF93EC018F8103
:100CA00090E001968F709927288530E0821793078E
:100CB00049F4CE010E940A06CE010E94ED05CE0144
:100CC0000E94D7052FB7F89498858F81891751F026
:100CD000FE01E90FF11D81859F5F9F709887C82FE6
:100CE000D0E002C0CFEFDFEF2FBFCF3F8FEFD807AD
:100CF00081F08091070480FF0CC0DF93CF938AEBD3
:100D000092E09F938F930E9451050F900F900F9048
:100D10000F90CE01DF91CF9108950F931F93CF9342
:100D20008C01CAE1C15071F0C8010E944C068F3F8E
:100D30002FEF920749F48FE99FE00197F1F700C088
:100D40000000F0CF8FEF9FEFCF911F910F9108958B
:100D50002F923F924F925F926F927F928F929F92CB
:100D6000AF92BF92CF92DF92EF92FF920F931F93B9
:100D7000CF93DF93EC01062F1B828091070480FF45
:100D80000CC01F926F938EEC92E09F938F930E9402
:100D900051050F900F900F900F908C819D818115C0
:100DA000904899F08091070480FF19C18C819D8142
:100DB0009F938F9384EC92E09F938F930E945105B1
:100DC0000F900F900F900F900AC19DB38B8D80955F
:100DD00089238DBB2BE0A22EBB24B39410E0992471
:100DE000939438E0232E47E0342E56E0452E65E0FC
:100DF000562E74E0872EE3E07E2EF2E06F2EA1ECFB
:100E0000CA2EA2E0DA2ECE010E94E1058FE193E026
:100E10000197F1F700C00000CE010E947A058FE132
:100E200093E00197F1F700C00000CE010E945A053F
:100E300068E97AE3CE010E94A505892B11F49B8213
:100E40006FC0E12CF12C90E59A95F1F7C8010E2CBA
:100E500002C0959587950A94E2F780FF05C0B924F2
:100E6000CE010E94850503C0CE010E947A0562E38F
:100E700070E0CE010E94BE05892B11F46B8250C038
:100E800062E370E0CE010E94A505892B11F47B82FC
:100E900047C02FEFE21AF20A88E0E816F10499F64B
:100EA00090E59A95F1F7CE01BB2019F00E948505D7
:100EB00002C00E947A0562E370E0CE010E94BE0586
:100EC000892B11F48B822CC062E370E0CE010E946A
:100ED000A505892B11F45B8223C020E52A95F1F743
:100EE000CE010E9485059CE2E92EFF24F394CE01F9
:100EF0000E949005882329F0E114F104C9F44B8283
:100F00000FC0EF28E1F38CE2E82EFF24F394CE012A
:100F10000E949005811114C0E114F104D1F53B82C7
:100F20008B81813009F049C0AA94A1103AC045C014
:100F300085E08A95F1F7000091E0E91AF108D7CF32
:100F4000EF2869F36CE271E0CE010E94BE05892BA7
:100F500011F42B82E5CFCE010E940A06CE010E9439
:100F6000D705CE010E94ED05CE01DF91CF911F91F3
:100F70000F91FF90EF90DF90CF90BF90AF909F9038
:100F80008F907F906F905F904F903F902F900C9438
:100F90008D0625E02A95F1F7000081E0E81AF108B6
:100FA000B6CF1B828091070480FF2DCFDF92CF92B6
:100FB0000E9451050F900F9026CF8B8180618B830B
:100FC000CE010E94E1058FE39FE10197F1F700C098
:100FD0000000CE010E94D705CE010E94ED058FEFE3
:100FE0009FEFDF91CF911F910F91FF90EF90DF90D6
:100FF000CF90BF90AF909F908F907F906F905F90B9
:101000004F903F902F9008951F93CF93DF93EC0163
:10101000162F6DEE0E94A8068A3F910539F4612FC4
:10102000CE01DF91CF911F910C94A806DF91CF9153
:101030001F9108951F920F920FB60F9211242F93B4
:101040003F934F935F938F939F93EF93FF9349B198
:101050005091B701909108042091A1013091A20113
:101060002115304819F49093A3010FC08091A3017A
:10107000981B933050F08091A1019091A201909320
:101080009E0180939D0180E21AC12091A1013091BF
:10109000A201369527953093A2012093A10181E00A
:1010A00090E001C0880F5A95EAF7842349F08091B7
:1010B000A1019091A20190689093A2018093A10157
:1010C0008091A1019091A20199278038910509F49E
:1010D00050C1A8F48032910509F44BC138F400974F
:1010E00009F447C1409709F495C0DEC080349105EA
:1010F00009F43FC18035910509F48CC0D5C0803C0E
:10110000910531F148F48039910509F483C0803AA2
:10111000910509F44DC0C8C0803D910509F47AC01D
:10112000803E910509F0C0C08091A1019091A2017B
:1011300090939E0180939D018091A1019091A201C5
:10114000892F99279093A2018093A10183E256C031
:1011500080919F01811123C084E629B19091B8014B
:10116000922311F48111EDC029B19091B80192231D
:10117000E1F08111ECC08091A1019091A2019093C6
:101180009E0180939D018091A1019091A201892FE0
:1011900099279093A2018093A10182E22FC08091B0
:1011A0009F01823209F0E5C0E6CF8111E2C0E3CFB2
:1011B00080919F01811125C084E629B19091B801E9
:1011C000922311F48111C9C029B19091B8019223E1
:1011D000F1F08111C8C08091A1019091A20190937A
:1011E0009E0180939D018091A1019091A201892F80
:1011F00099279093A2018093A10181E280939F019E
:101200006BC080919F01813209F0B3C0E4CF81119E
:10121000B0C0E1CF8091A1019091A20190939E0175
:1012200080939D018091A1019091A20180399A4AF9
:1012300011F482E044C02091A1013091A20180917B
:10124000A1019091A20124E0329F212D3327112486
:10125000217056E0969587955A95E1F78227982F49
:101260009E7F29F0982F969581708927F8CF81115C
:1012700002C081E024C08091A1019091A20197FF5A
:1012800002C080E101C081E180939F018091A101B2
:101290009091A20126E0969587952A95E1F7909383
:1012A000A2018093A10118C010929F018091A10119
:1012B0009091A20190939E0180939D0180E880937C
:1012C000A0019BB18091B801282F209592239BB952
:1012D0009AB1892B8AB92EC02091A1013091A20127
:1012E0008091A401E82FF0E0E356FE4F21878F5F45
:1012F0008F708093A40190E001968F7099273091B0
:10130000A501432F50E08417950769F42DB3809110
:10131000B801482F409524232DBB9BB194239BB942
:101320009AB1892B8AB98091A401831303C080E408
:101330008093A00180E090E89093A2018093A101A6
:1013400018C095E09A95F1F70000815006CF25E08E
:101350002A95F1F70000815007CF95E09A95F1F7B3
:10136000000081502ACF25E02A95F1F70000815036
:101370002BCFFF91EF919F918F915F914F913F9173
:101380002F910F900FBE0F901F9018951F920F92E4
:101390000FB60F9211242F933F934F935F938F9328
:1013A0009F93EF93FF9349B150919A019091080454
:1013B00020918401309185012115304819F49093D2
:1013C00086010FC080918601981B933050F0809168
:1013D000840190918501909381018093800180E246
:1013E0001AC120918401309185013695279530935B
:1013F00085012093840181E090E001C0880F5A9517
:10140000EAF7842349F080918401909185019068E6
:10141000909385018093840180918401909185014E
:1014200099278038910509F450C1A8F480329105BC
:1014300009F44BC138F4009709F447C1409709F407
:1014400095C0DEC08034910509F43FC18035910517
:1014500009F48CC0D5C0803C910531F148F4803945
:10146000910509F483C0803A910509F44DC0C8C0C4
:10147000803D910509F47AC0803E910509F0C0C015
:1014800080918401909185019093810180938001E6
:101490008091840190918501892F992790938501EE
:1014A0008093840183E256C080918201811123C020
:1014B00084E629B190919B01922311F48111EDC032
:1014C00029B190919B019223E1F08111ECC08091B0
:1014D0008401909185019093810180938001809196
:1014E000840190918501892F99279093850180939C
:1014F000840182E22FC080918201823209F0E5C02E
:10150000E6CF8111E2C0E3CF80918201811125C035
:1015100084E629B190919B01922311F48111C9C0F5
:1015200029B190919B019223F1F08111C8C0809163
:101530008401909185019093810180938001809135
:10154000840190918501892F99279093850180933B
:10155000840181E2809382016BC08091820181329B
:1015600009F0B3C0E4CF8111B0C0E1CF8091840114
:1015700090918501909381018093800180918401F5
:101580009091850180399A4A11F482E044C02091FB
:10159000840130918501809184019091850124E03E
:1015A000329F212D33271124217056E0969587957F
:1015B0005A95E1F78227982F9E7F29F0982F9695CC
:1015C00081708927F8CF811102C081E024C0809109
:1015D00084019091850197FF02C080E101C081E103
:1015E00080938201809184019091850126E09695F7
:1015F00087952A95E1F7909385018093840118C01F
:1016000010928201809184019091850190938101D3
:101610008093800180E8809383019BB180919B013E
:10162000282F209592239BB99AB1892B8AB92EC075
:10163000209184013091850180918701E82FF0E0AD
:10164000E058FE4F21878F5F8F708093870190E075
:1016500001968F70992730918801432F50E08417AD
:10166000950769F42DB380919B01482F4095242361
:101670002DBB9BB194239BB99AB1892B8AB98091D8
:101680008701831303C080E48093830180E090E8A6
:10169000909385018093840118C095E09A95F1F7A5
:1016A0000000815006CF25E02A95F1F70000815017
:1016B00007CF95E09A95F1F7000081502ACF25E0F9
:1016C0002A95F1F7000081502BCFFF91EF919F9168
:1016D0008F915F914F913F912F910F900FBE0F907F
:1016E0001F901895EDE9F1E01182108212821382A9
:1016F00020E030E835832483168291E0918F128EAA
:1017000082E0838F948FE0E8F1E0118210821282F0
:10171000138235832483168293E0918F828F88E031
:10172000838F84E0848F0895262F30E094E03595F0
:1017300027959A95E1F72770E62FEF70823069F0D0
:101740008330A1F08130E1F4F0E080E1289FE00DEA
:10175000F11D1124E85AFA4F11C0F0E080E1289FF2
:10176000E00DF11D1124E852FB4F08C0F0E080E1CC
:10177000289FE00DF11D1124E85AFB4F8491089534
:1017800080E808950F931F93CF93DF938C01EB01B3
:1017900069EEFC01808191810E94A806F801808198
:1017A00091810E948D068883F801808191810E9439
:1017B0008D068983F801808191810E948D068A833C
:1017C00099279F938F9389811F928F9388811F926E
:1017D0008F9385E494E09F938F930E9451058DB77A
:1017E0009EB708960FB6F8949EBF0FBE8DBFDF91CF
:1017F000CF911F910F910895E7EDF1E011921192B1
:1018000081E0E73EF807D1F70895CF93DF93EC012D
:101810001B821A821C821D820E94FC0B8881998186
:10182000DF91CF910C9416061F93CF93DF93FC01A9
:1018300084810E94940B87FD20C0182F1F70C82F31
:10184000D0E094E0D595C7959A95E1F7612F8C2F5C
:101850000E94E021811111C0CC0FDD1FC952DE4F63
:1018600081E090E002C0880F991F1A95E2F7288165
:101870003981822B932B99838883DF91CF911F919C
:1018800008951F93CF93DF93FC0184810E94940BF2
:1018900087FD22C0182F1F70C82FD0E094E0D59587
:1018A000C7959A95E1F7612F8C2F0E94E02188233C
:1018B00099F0CC0FDD1FC952DE4F81E090E002C0ED
:1018C000880F991F1A95E2F78095909528813981A4
:1018D0008223932399838883DF91CF911F91089569
:1018E00089EC91E00E94050C8BEB91E00C94050CC7
:1018F000809107048160809307040C94FC0BE82F0F
:10190000F0E0EE0FFF1FE952FE4F808191810895B4
:101910000C94FC0B7770E72FF0E098E0899FE00DC6
:10192000F11D112484E0EE0FFF1F8A95E1F76F701F
:10193000E60FF11DEE0FFF1FE050F84985919491DD
:1019400008958091BA010895FC018481823070F07D
:10195000843061F062FB992790F960FD926061FD2F
:101960009460692F808191810C9404080895CF932D
:10197000C82F682F89EC91E00E94A40C6C2F8BEB90
:1019800091E0CF910C94A40CCF92DF92EF92FF9252
:101990000F931F93CF93DF936C018B010E94072E4F
:1019A0007C01F601808191810E944C06EC01019638
:1019B00031F4C7010E941F2E8017910790F3CE01CA
:1019C000DF91CF911F910F91FF90EF90DF90CF901B
:1019D00008950F931F93CF93DF93FC018081918132
:1019E000DC0112962C912131F9F08F0162EF0E94F7
:1019F000A8068F3FBFEF9B07D1F08A3F9105D1F436
:101A000064EF71E0C8010E94C40C8F3F2FEF920772
:101A1000A1F0D82FCC2764EF71E0C8010E94C40C5C
:101A2000DE01A82BCD010BC08DEF9FEF08C08FEF1B
:101A30009FEF05C08EEF9FEF02C080E090E0DF9146
:101A4000CF911F910F910895CF93862F90E0FC01C5
:101A50007C97E834F105A0F5EA5AFF4F0C946C32FC
:101A600085E53EC08AE53CC08BE53AC08CE538C0D0
:101A70008DE536C08EE534C08FE532C080E630C0DB
:101A800081E62EC082E62CC083E62AC08FE628C0FD
:101A900081E726C082E724C084E722C085E720C012
:101AA00087E71EC088E71CC08AE71AC08CE718C009
:101AB0008FE716C080E714C089E712C08BE710C01B
:101AC000C62F1F926F938BE293E09F938F930E9498
:101AD00051050F900F900F900F908C2F01C084E54F
:101AE000CF910895CF93DF93EC0199859230A9F1BE
:101AF00028F4992341F09130C9F045C09330B1F1F9
:101B00009430D9F140C0603E21F0613E21F482E082
:101B10002BC081E029C067FD04C0CE010E94140CD7
:101B200033C06F77CE010E94410C2EC0663359F14D
:101B300018F46A3229F427C06A3A29F1663B19F190
:101B400067FD05C0CE010E94240D682F12C06F777B
:101B5000CE010E94240D682F13C06D3121F06D3924
:101B600091F484E001C083E089870EC0653459F4A4
:101B700065E5CE010E94140C06C0653C21F465E5C4
:101B8000CE010E94410C198680E0DF91CF9108952B
:101B9000862F90E0FC013397E138F10508F048C04A
:101BA000E256FF4F0C946C3289E1089587E1089565
:101BB0008FE1089587E2089580E6089582E608950A
:101BC0008CE5089583E508958FE2089589E30895EB
:101BD00087E308958FE3089587E408958FE40895D7
:101BE00086E508958EE508958FE7089580E00895CD
:101BF00085E608958EE608958FE6089580E30895BA
:101C000088E3089580E4089588E4089580E50895C0
:101C100087E508958FE5089588E1089588E008959F
:101C200080E2089580E108958DE6089588E20895A0
:101C3000862F8F7708958FE00895623309F44AC0A4
:101C400010F5643209F44CC080F46C3109F44CC0D6
:101C500028F46B3109F04AC08FE108956D31F1F13C
:101C6000633209F043C087E208956B3209F440C043
:101C700020F46A32D9F588E408956C3229F16D3286
:101C8000A9F581E508956234E9F048F46433B1F0D0
:101C9000B8F06A3309F16C3349F580E308956B3489
:101CA000B9F030F4633491F0643401F585E60895B9
:101CB0006D34C1F06136D1F48AE6089580E108956B
:101CC00088E1089580E2089588E2089588E3089500
:101CD00080E4089580E5089587E508958FE50895E7
:101CE00087E108958EE608958FE60895862F08957A
:101CF00088E008956B35C9F068F46131F1F020F4A3
:101D00006E30C9F484E50895633169F0643599F45F
:101D10008BE508956D3559F050F0623651F06C370F
:101D200051F487E7089581E108958DE508958AE6E5
:101D300008958EE00895862F08958FE0089561310B
:101D400031F0613411F48CE70895862F089583E112
:101D500008951F93CF93DF93EC01162FEA858E2F02
:101D600090E08B30910508F0D2C0FC01E15EFE4F9F
:101D70000C946C328A819B8180599B4A029720F493
:101D8000CE010E947A0E182F1438A9F030F41038C2
:101D900081F0133891F462E090C0113E41F0103FA1
:101DA00021F0103E51F482E08FC081E08DC084E0CC
:101DB0008BC089E089C06FE780C01A8617FD02C01A
:101DC000612F98C00E94FC0B8FE193E063C08A8171
:101DD0009B8180599B4A029720F4CE010E949F0E5E
:101DE000182F193509F493C0103F19F0123119F466
:101DF0008EC083E069C01A8617FD05C0612FCE0131
:101E00000E94C80D76C00E94FC0B85E193E042C0A1
:101E10008A819B8180599B4A029720F4CE010E94BF
:101E20007A0E182F133821F0143821F46FE755C0BB
:101E300062E053C01A8617FD02C0612F64C00E9481
:101E4000FC0B1F921F9386E093E09F938F930E9459
:101E500051050F900F900F900F9022C08A819B81A7
:101E600080599B4A029720F4CE010E949F0E182FA2
:101E70001A86123109F44CC0193509F449C017FD0E
:101E800005C0612FCE010E94C80D3CC00E94FC0B12
:101E900089EF92E09F938F930E9451050F900F90CE
:101EA0008FEF37C0643121F0603F89F586E00CC0C8
:101EB00085E00AC0673759F560E0CE010E94140C36
:101EC00026C0643121F587E08A8722C0603FF9F49B
:101ED00088E0FACF6737D9F460E0CE010E94410C68
:101EE00016C0603F11F48AE0EFCF1A86CE010E943F
:101EF0001D0E682FCE010E94140C0AC01A86CE0156
:101F00000E941D0E682FCE010E94410C01C01A864E
:101F100080E0DF91CF911F9108956C3551F018F456
:101F2000633169F00AC0663731F06E3731F486E705
:101F3000089581E508958EE70895862F08958DE52B
:101F40000895663809F466C058F5673609F450C03C
:101F5000A0F46C3509F464C040F4683009F464C03E
:101F6000673509F05FC08CE50895643609F444C014
:101F7000653609F057C08DE60895673709F44EC0FD
:101F800038F46D36B9F16E3609F04CC085E6089527
:101F90006438A1F1E8F56C3709F044C088E608958B
:101FA0006C38A1F178F4693869F130F4673841F19F
:101FB0006838C1F58EE708956A3831F16B3891F5CC
:101FC00084E008956F3881F030F46D3859F06E3840
:101FD00049F587E608956139F9F040F0623911F565
:101FE00089E0089587E708958FE708958BE70895BE
:101FF00082E6089584E608958EE608958CE70895B4
:1020000082E008958CE0089583E0089585E00895C6
:1020100088E0089580E1089581E0089588E50895B5
:1020200083E50895862F089586E70895CF93DF937B
:10203000EC016F3B41F028F486E5860F823070F4A6
:1020400002C06C3F59F41B868CEE92E09F938F93F5
:102050000E9451050F900F908FEFC1C08B8581308A
:1020600009F44DC038F0823009F486C0833009F499
:10207000A1C0B4C08A819B8182392BEA920721F4E6
:10208000CE010E948D0F06C081399B4A21F4CE01FA
:102090000E94A10F682F663809F168F46338D1F007
:1020A00020F4603819F582E07FC06438A9F0653803
:1020B000E9F468E61DC06C38A9F030F4673881F0A7
:1020C0006B38A1F461E014C06D3871F0603F71F4B9
:1020D00081E06AC062E00CC06FE70AC068E708C030
:1020E00060E006C069E004C06AE002C067FD04C0A9
:1020F000CE010E94140C72C08FED92E036C01B8698
:102100008A819B8182392BEA920721F4CE010E94B9
:102110008D0F06C081399B4A21F4CE010E94A10F88
:10212000682F862F90E0FC01E358F109EB30F105B0
:10213000A0F4E65DFE4F0C946C3262E010C06FE7D5
:102140000EC068E60CC068E70AC060E008C061E045
:1021500006C069E004C06AE002C067FD04C0CE01A9
:102160000E94410C3BC085ED92E09F938F930E94AB
:1021700051050F900F9032C0653279F030F466311E
:1021800071F06E3199F460E00BC0663221F0603F6F
:1021900069F483E009C06DE503C063E501C061E552
:1021A000CE010E94140C04C08B8718C00E94FC0B47
:1021B0001B8614C06E3169F020F46631B9F761E511
:1021C00009C0653221F0663289F76DE503C063E529
:1021D00001C060E0CE010E94410CEACF80E0DF91B7
:1021E000CF9108958F929F92AF92BF92CF92DF923C
:1021F000EF92FF920F931F93CF93DF9300D000D005
:102200001F92CDB7DEB78C01DC01ED91FC9183818B
:10221000882391F1E080F180D3800E94072EFF9205
:10222000EF921F92DF929F938F938EE294E09F93A1
:102230008F930E945105D801ED91FC9111978381F4
:1022400080750FB6F894DEBF0FBECDBF79F4189637
:102250008C9118978B3019F48CE018968C938381AD
:10226000823021F48DE0D80118968C931382D80126
:10227000ED91FC9111821082D801ED91FC911197A2
:102280008281882381F1928115968C91981759F15A
:10229000E080F180D2800E94072EFF92EF921F9281
:1022A000DF929F938F9387E194E09F938F930E9497
:1022B0005105F80185810FB6F894DEBF0FBECDBF82
:1022C0000190F081E02D85FF03C0928194FDA1C5AE
:1022D00084FD9CC5D801ED91FC91119782811596E2
:1022E0008C9311821082D8011896EC918E2F90E079
:1022F0008E30910508F0E9C5FC01EB5CFE4F0C94B3
:102300006C320E94072E9F938F938BE094E09F93F3
:102310008F930E9451050E94072EF80197838683B0
:10232000808191810E94F70581E0D80118968C93F5
:102330006BC0F801808191810E944C060196C9F71B
:10234000D80116968D919C9117970E941F2E893B5C
:102350009B4008F4BAC582E041C50E94072E9F93B6
:102360008F9386E094E09F938F930E9451056FEFC7
:10237000D8018D919C910E94A8060F900F900F900C
:102380000F908A3F910511F486E028C583E06FC362
:10239000F801808191810E9401062E98269A2F983B
:1023A000279A0E94072ED80117969C938E93169712
:1023B00084E05EC3F801868197810E941F2E853FCD
:1023C000914008F482C585E052C32E9826982F9834
:1023D0002798F801808191810E940A06D8018D9189
:1023E0009C910E94F7050E94072E9F938F9381E096
:1023F00094E09F938F930E9451050E94072EF8014D
:102400009783868386E080870F900F900F900F90C0
:102410005CC5D8018D919C910E944C06019609F4EF
:1024200054C50E94072E9F938F938CEF93E09F9348
:102430008F930E9451050E94072EF801978386838F
:1024400087E0E1CFD80116968D919C9117970E9455
:102450001F2E853F914018F089E0F8018087D80150
:102460008D919C910E944C06019609F42EC50E9404
:10247000072E9F938F9387EF93E09F938F930E94F4
:1024800051050E94072EF8019783868388E0BBCF11
:10249000D80116968D919C9117970E941F2E853F0B
:1024A000914018F089E0F8018087D8018D919C91C6
:1024B0000E944C06019609F408C50E94072E9F93BE
:1024C0008F9382EF93E09F938F930E94510589E051
:1024D000F80199CFC8010E94E90CD80113969C938A
:1024E0008E9312970E94072E9F938F938DEE93E009
:1024F0009F938F930E945105F801828193810F90E1
:102500000F900F900F90009711F482E010C08F3F52
:10251000BFEF9B0711F481E044C09C012D5F3F4F4A
:102520002230310590F38F3F910529F484E0D801E2
:1025300014968C9372C09C0125583B4A2230310579
:1025400008F49FC48239BBEA9B0709F49AC49C0132
:1025500020593B4A22303105F8F480EE93E09F93F6
:102560008F930E94510582E0F801848360EF80819F
:1025700091810E94A8060F900F908A3F9105F1F576
:1025800062E8D8018D919C910E94A8068A3F91052E
:10259000A9F58CED93E06EC4803BBFEB9B0721F463
:1025A00083E0F801848339C088278115FBEA9F07FF
:1025B00009F4ABCF81152FEB920791F381159F475B
:1025C00079F384EB93E09F938F930E94510560EF22
:1025D000D8018D919C910E94A8060F900F908A3F80
:1025E000910509F04EC462E0F801808191810E945A
:1025F000A8068A3F910509F044C487CF88ED93E08F
:102600009F938F930E9451050F900F90F801828144
:10261000938181399B4A09F40EC4F80122813381E8
:102620002E3FFFEF3F0751F02D3F4FEF340749F0AA
:102630002115310549F040E251E008C041E251E086
:1026400005C04BE151E002C047E251E0D8011496C9
:102650008C91813049F0823051F0833059F08430D0
:1026600061F08CE391E00BC080E391E008C08DE263
:1026700091E005C083E391E002C081E491E05F93C3
:102680004F939F938F933F932F9384EA93E09F936D
:102690008F930E9451058AE0F801808781C30E94D0
:1026A000072E9F938F938FE993E09F938F930E94C0
:1026B00051050F900F900F900F90D80114968C91A8
:1026C000833031F0843079F0823009F07CC106C06B
:1026D00068EFF801808191810E94A8060E944C2039
:1026E0000E94B70C70C165EFD8018D919C910E943A
:1026F000A8066AEEF801808191810E94A806BE01B9
:102700006F5F7F4FC8010E94C20B88E993E09F93DF
:102710008F930E94510568EED8018D919C910E9483
:10272000A80660E0F801808191810E94A80666EE0B
:10273000D8018D919C910E94A80666EEF8018081D7
:1027400091810E94A80666EED8018D919C910E940D
:10275000A806BE016F5F7F4FC8010E94C20B0F9099
:102760000F908981882309F47AC08A81882309F42B
:1027700076C081E993E09F938F930E94510566EEA6
:10278000F801808191810E94A80668EED8018D91A0
:102790009C910E94A80660E0F801808191810E94CE
:1027A000A80668EED8018D919C910E94A80663E06E
:1027B000F801808191810E94A80668EED8018D9170
:1027C0009C910E94A80662E0F801808191810E949C
:1027D000A80668EED8018D919C910E94A80661E040
:1027E000F801808191810E94A80666EED8018D9142
:1027F0009C910E94A80668EEF801808191810E9458
:10280000A80663E0D8018D919C910E94A80668EE0D
:10281000F801808191810E94A80661E0D8018D9124
:102820009C910E94A80668EEF801808191810E9427
:10283000A80662E0D8018D919C910E94A80668EEDE
:10284000F801808191810E94A80663E0D8018D91F2
:102850009C910E94A80689E0F801848781C08AE8DB
:1028600093E09F938F930E94510563EFD8018D9160
:102870009C910E94A80668ECF801808191810E94D9
:10288000A80663EFD8018D919C910E94A80664E68A
:10289000F801808191810E94A80663EFD8018D9193
:1028A0009C910E94A80660E5F801808191810E94B8
:1028B000A806C8010E94E90C292F30E00F900F9064
:1028C0002330310511F080E001C083E0D8011C966F
:1028D0008C9383E893E09F938F930E94510563EF5D
:1028E000F801808191810E94A80668ECD8018D9141
:1028F0009C910E94A80663EFF801808191810E945B
:10290000A80668ECD8018D919C910E94A80663EFFF
:10291000F801808191810E94A80660E5D8018D911F
:102920009C910E94A806C8010E94E90C292F30E062
:102930000F900F902430310511F080E001C084E049
:10294000F801848781110EC08CE793E09F938F93E9
:102950000E94510566EFD8018D919C910E94A806B6
:102960000F900F9064EFF801808191810E94A8067A
:10297000BE016F5F7F4FC8010E94C20BD8011C9639
:102980008C91893049F0833051F0843059F088239C
:1029900061F083E291E00BC08FE491E008C087E42E
:1029A00091E005C088E591E002C081E691E09F9347
:1029B0008F9380E793E09F938F930E9451050F9030
:1029C0000F900F900F908BE0F80180870E94072EE8
:1029D0009F938F938BE693E09F938F930E94510573
:1029E0000F900F900F900F90D8018D919C910E94A5
:1029F0004C064C01019609F468C2F80184818430C8
:102A000069F18114910421F0FFEF8F16910469F4AC
:102A10000E94FC0B0E94762383E693E09F938F93A2
:102A20000E9451050F900F9050C2823069F08330A0
:102A300081F0813009F049C2682DC8010E94720DF1
:102A40008F3F09F042C212C0682DC8010E94A90E32
:102A5000F7CF682DC8010E941610F2CFF8018081CF
:102A600091810E948D066C01019629F48CE0D801B9
:102A700018968C932AC2F801808191810E948D065C
:102A80007C01019699F3D8011C968C91FE01319638
:102A90005F01853028F4833030F4882321F0DEC0D4
:102AA0008930A1F0DBC0D8011D969C911D97987FBD
:102AB000282D2770922B1D969C9384FE02C0DD2446
:102AC000DA9485FEC6C0FF24FA94C3C0F8013585A8
:102AD000C401887499278834910509F0ABC0C1FE00
:102AE000A9C0F0E38F2299249594879495948794B4
:102AF00020E3C222DD2454E0D594C7945A95E1F72F
:102B0000C828D92842E0C416D104E1F183E0C816F0
:102B1000D10409F478C0CA94CD2809F0C7C1E6FCF5
:102B200017C0A701487055278E2D8F70E7FE07C08C
:102B3000452B11F420E001C020EF822B0AC0452B69
:102B400011F420E001C020EF982F922B80E002C00A
:102B500080E090E0E4FE05C03860D8011D963C930B
:102B600003C0377FF8013587D8011D962C911D973A
:102B7000E5FE04C020611D962C939AC12F7EF801BA
:102B8000258796C1E0FE05C03064D8011D963C93B0
:102B900003C03F7BF8013587D8011D968C911D97A6
:102BA000E1FE04C080681D968C9303C08F77F80106
:102BB0008587D8011D968C911D97E2FE04C0806226
:102BC0001D968C9303C08F7DF8018587D8011D96D3
:102BD0008C911D97E3FE04C080641D968C9303C006
:102BE0008F7BF8018587D8011D968C911D97E4FE97
:102BF00004C080681D968C9303C08F77F801858789
:102C000080E090E055C1C70124E0959587952A950D
:102C1000E1F7E7FE03C0806F90E003C0982F9F703C
:102C200080E0387F2E2D2770E32EE22AD8011D96F2
:102C3000EC923EC1387F882D8770382BF80135879C
:102C400084FE02C0DD24DA9485FE4DC0FF24FA9490
:102C50004AC0833049F08430C9F045C0833079F4EC
:102C6000E12CF12CC12CD12CD8018D919C910E948A
:102C70008D068F3FBFEF9B07B1F1982F35C0843091
:102C800009F014C1E12CF12CC12CD12CF801808168
:102C900091810E948D06AC018F3FFFEF9F0719F1D4
:102CA00083FD02C080E001C080EF942F9F70982BBD
:102CB000D8011D962C911D9744FF04C028601D96D5
:102CC0002C9303C0277FF8012587D8011D962C91EE
:102CD0001D9745FF04C020611D962C9305C02F7ED3
:102CE000F801258701C090E085E0D5011D928A9505
:102CF000E9F7F8018585898380E0F0E8CF16D104F3
:102D00004CF4960141E8C4164FEFD40624F421E8B0
:102D10003FEF01C02FE72A83A0E8EA16F10454F43C
:102D20009701B1E8EB16BFEFFB0614F421E83FEF83
:102D3000219501C021E82B83903811F0919501C0B5
:102D40009FE79C83803809F481E88D83C5010E9448
:102D5000A12089818093BA011F928F938D81282FA2
:102D6000082E000C330B3F938F938C81282F082E55
:102D7000000C330B3F938F938B81282F082E000C70
:102D8000330B3F938F938A81282F082E000C330B2F
:102D90003F938F9384E493E09F938F930E94510518
:102DA0000FB6F894DEBF0FBECDBF8FC00E94072EB6
:102DB0009F938F938FE393E09F938F930E9451058E
:102DC0006EEFD8018D919C910E94A8060F900F90F4
:102DD0000F900F908A3A910521F489E0F8018087DD
:102DE00074C00E94072E9F938F938AE393E09F9372
:102DF0008F930E945105C8010E94050C0E94FC0B94
:102E00000E947623D80118961C92FECA828185FF03
:102E100061CAD80118968C918B3009F05BCA80E1A9
:102E200094E09F938F930E9451058CE0F801808776
:102E30000F900F904FCA60EFF801808191810E943E
:102E4000A8068A3F9105A1F463E0D8018D919C9179
:102E50000E94A8068A3F910559F484ED93E09F9360
:102E60008F930E94510583E0D80114968C9306C07D
:102E700080ED93E09F938F930E9451050F900F90E8
:102E8000CCCB60EFF801808191810E94A8068A3F37
:102E9000910509F03ACB63E0D8018D919C910E9495
:102EA000A8068A3F910509F030CB7ACB90E080E00C
:102EB00025E0D5011D922A95E9F7F801258529839A
:102EC000E12CF12CC12CD12C1CCF81E00F900F9064
:102ED0000F900F900F90DF91CF911F910F91FF9066
:102EE000EF90DF90CF90BF90AF909F908F9008951C
:102EF00089EC91E00E94F2108BEB91E00C94F210BF
:102F0000E9ECF1E08DE991E09183808313821282F4
:102F100014821582108611861286138614861586F1
:102F20000E94FC0BEBEBF1E080E891E09183808361
:102F300013821282148215821086118612861386DD
:102F4000148615860C94FC0B80910B030895CF9387
:102F5000DF9300D01F92CDB7DEB720911904243043
:102F600021F523E029839B838A8382E08093E90013
:102F70008FEF9091E800815095FD06C095ED9A95F0
:102F8000F1F700008111F5CF8091E80085FF0DC0B9
:102F900040E050E063E070E0CE0101960E94771CB3
:102FA0008091E8008E778093E8000F900F900F904B
:102FB000DF91CF910895CF93DF9300D01F92CDB7CB
:102FC000DEB720911904243061F519821A821B8220
:102FD00022E029838138910520F0805891099B8354
:102FE0008A8382E08093E9008FEF9091E80081501E
:102FF00095FD06C095ED9A95F1F700008111F5CF8A
:103000008091E80085FF0DC040E050E063E070E093
:10301000CE0101960E94771C8091E8008E77809304
:10302000E8000F900F900F90DF91CF9108952091BD
:103030001904243051F522E02093E9002FEF30915C
:10304000E800215035FD06C035ED3A95F1F7000056
:103050002111F5CF2091E80025FF17C02091100124
:10306000222341F021E02093F10040E050E065E0B0
:1030700070E004C040E050E063E070E00E94771C24
:103080008091E8008E778093E8000895CF93DF93D6
:1030900020911904243009F04AC0EC0180911101FB
:1030A0008823E1F0809112018823C1F081E08093B0
:1030B000E90081E8815049F09091E80095FD05C054
:1030C0009AE29A95F1F700C0F5CF8091E80085FF6C
:1030D0002EC040E050E060E270E019C081E08093D3
:1030E000E90081E8815059F09091E80095FD07C012
:1030F000EFE3F1E03197F1F700C00000F3CF8091EA
:10310000E80085FF14C040E050E068E070E0CE01C8
:103110000E94771C8091E8008E778093E80080E21F
:10312000FE01ABEEB2E001900D928A95E1F7DF91DE
:10313000CF910895CF93C091E901C1110BC00E94B6
:10314000132E643C79408105910520F081E0809345
:10315000E901C1E08C2FCF910895FF920F931F9347
:10316000CF93DF93D82F0FB607FE83C08091190449
:10317000843081F08091030190E001962091050157
:1031800030E0822393232091040130E082179307DB
:1031900009F0CDC00E949A18811110C080910301DE
:1031A00090E001962091050130E082239323209145
:1031B000040130E08217930709F0B9C00E94072E7E
:1031C0008C01C091E900CF709091EC00892F817043
:1031D00090FD80E8C82B83E08093E90085E0F82E1D
:1031E0008091EB0085FD42C08091EB0080FF3EC0E6
:1031F0008091EE0087FF3AC0809104019091030115
:10320000981709F457C09091E80095FF8EC0E0919F
:103210000101F0910201E80FF11D20818F5F909173
:1032200005018923809304012093F1008091E80037
:1032300085FDE2CF8091E80080FFDECF8091E8003D
:103240008E778093E800F0920001D6CF8091030141
:1032500090E001962091050130E082239323209194
:10326000040130E08217930709F44CC0CF70C0937B
:10327000E90040910301842F90E00196209105011F
:1032800030E0822393232091040130E082179307DA
:1032900009F450C0E0910101F0910201E40FF11D29
:1032A000D083809103018F5F9091050189238093E2
:1032B000030140C08091E80085FF37C0D093F10042
:1032C00021E03091F3008091F20090E0932B892B64
:1032D00091F08091E80080FF0EC08091E80085FFAA
:1032E00003C01092F100F9CF8091E8008E778093AF
:1032F000E800F0920001222309F4A8CFCF70C09318
:10330000E90018C080910001882309F4AFCF0E9422
:10331000072E9C018017910711F4890161CF9091CC
:103320000001915090930001F8CF20E0CACF409166
:103330000301B0CF80E0DF91CF911F910F91FF90FB
:10334000089580911804811104C00E94E31E0C941A
:10335000401F0895109218040895089542E261EC08
:1033600081E00E94F01B42E061EC82E00E94F01BD1
:1033700042E261EC83E00C94F01B80911B048330EB
:1033800009F453C030F4813071F0823009F4BAC0CE
:1033900008958A3009F4A6C08B3009F478C08930CA
:1033A00009F0C8C020C080911A04813A09F0C2C057
:1033B0008091E800877F8093E80080911E049091BF
:1033C0001F04892B21F460E28BEE92E003C060E0E1
:1033D00080E090E070E00E94C41C8091E8008B7750
:1033E0008093E800089580911A04813209F0A2C008
:1033F00080911E0490911F04892B09F09BC080913D
:10340000E800877F8093E8008091E80082FD05C096
:10341000809119048111F8CF8DC08091F1008093C3
:103420000B038091E8008B7781C080911A04813A68
:1034300009F080C080911E0490911F04892BA1F493
:103440008091E800877F8093E8008091E80080FF0A
:10345000FCCF809111018093F1008091E8008E777C
:103460008093E8000E94251C80911E0490911F0407
:10347000019709F05FC08091E800877F8093E800A2
:103480008091E80080FFFCCF809110014AC08091BC
:103490001A04813209F04EC080911E0490911F04DD
:1034A000892B69F48091E800877F8093E8000E946F
:1034B000251C80911C04809311010E947623809129
:1034C0001E0490911F040197A9F58091E800877F61
:1034D0008093E8000E94251C80911C0480931001B9
:1034E0000C94762380911A04813221F58091E800B2
:1034F000877F8093E8000E94251C80911D048093A3
:103500000C03089580911A04813AA1F48091E80097
:10351000877F8093E8008091E80080FFFCCF809156
:103520000C038093F1008091E8008E778093E8008F
:103530000C94251C089580910B038093EA0110924E
:103540000B030E94880C0C9476230C949B1A0E9407
:10355000B32D80911704882329F00E94C02D81117A
:103560000C94DA1B08950E94D52D8091EA01809376
:103570000B0308950C94B31A08950C94BC1ACF93BE
:1035800084B7877F84BF0FB6F894A89580916000B8
:10359000886180936000109260000FBE90E080E828
:1035A0000FB6F89480936100909361000FBE8DEA8E
:1035B00098E10E94722D86E091E00E94472088EFFA
:1035C00095E00E94B8040E94700C0E941E210E9487
:1035D000E31E0E94401F78940E94202180911904CC
:1035E000843029F00E942C200E94BC1AF7CF86EE6E
:1035F00095E00E94B8040E94BD1A88ED95E00E94F3
:10360000B804C3E080911904853019F40E94A71A08
:10361000F9CF0E949C2D0E9424212091E40030913A
:10362000E5008091E7019091E8012817390709F436
:1036300068C08091E4009091E5009093E801809348
:10364000E7010E949A18882309F45BC0809119044D
:10365000843009F056C08091E9008F702091EC0011
:10366000922F917020FD90E8892BC093E9009091F2
:10367000EB0090FF43C09091EE0097FF3FC0909108
:10368000040120910301291709F12091E80025FF89
:103690001DC0E0910101F0910201E90FF11D30819F
:1036A0009F5F209105019223909304013093F100D4
:1036B0009091E80095FDE3CF9091E80090FFDFCF77
:1036C0009091E8009E779093E800D9CF9091F30015
:1036D0002091F20030E0392B232B81F09091E8000B
:1036E00090FF0CC09091E80095FF03C01092F1008C
:1036F000F9CF9091E8009E779093E8008F708093C7
:10370000E9000E942C207ECF292F3327233031055A
:10371000C9F060F42130310581F02230310509F023
:1037200041C084E590E025E536E040C02132310516
:10373000E1F02232310531F135C082E190E029EA31
:1037400036E034C099278130910549F028F002977E
:1037500049F5E1E1F6E005C0E1E5F6E002C0E7E4A5
:10376000F6E0849190E09F0121C063307105D0F4B0
:10377000660F771FFB01EE58FE4F2081318189E0F3
:1037800090E014C06330710568F4FB01EE0FFF1F79
:10379000E459FE4F20813181FB01E759FE4F8081C2
:1037A00090E004C080E090E020E030E0FA01318356
:1037B0002083089580E189BD82E189BD09B400FEBE
:1037C000FDCF8091D8008F7D8093D8008091E0005C
:1037D00082608093E0008091E00081FDFCCF08953D
:1037E000982F973068F59093E900981739F0709109
:1037F000EC002091ED005091F00003C0242F762FB3
:1038000050E021FD02C09F5FECCF3091EB003E7F86
:103810003093EB003091ED003D7F3093ED0030911F
:10382000EB0031603093EB007093EC002093ED00DF
:103830005093F0002091EE0027FDE5CF80E0089541
:103840008F708093E90081E0089580911A0487FFCA
:1038500011C08091E80082FD05C08091190481119A
:10386000F8CF11C08091E8008B770BC080911904CC
:10387000882349F08091E80080FFF8CF8091E8002C
:103880008E778093E80008952091E4003091E50060
:1038900095E64091EC00842F817040FF23C0809119
:1038A000E80080FD1DC080911904882399F08530BF
:1038B00099F08091EB0085FD11C04091E40050919A
:1038C000E5002417350729F3915011F09A01E1CF53
:1038D00084E0089582E0089583E0089581E00895EA
:1038E00080E008954091E80042FFDDCF0895CF9237
:1038F000DF92EF92FF920F931F93CF93DF93EC0130
:103900008B017A010E94441C811135C0E114F1043D
:1039100039F0F70180819181081B190BC80FD91F5D
:10392000C12CD12C0115110529F18091E80085FDEC
:1039300018C08091E8008E778093E8000E942C20C8
:10394000E114F10449F0F70180819181C80ED91E7C
:10395000D182C08285E00FC00E94441C882311F3ED
:103960000AC089918093F10001501109FFEFCF1A2D
:10397000DF0AD8CF80E0DF91CF911F910F91FF90A8
:10398000EF90DF90CF900895209120043091210492
:103990002617370748F06115710539F42091E800C2
:1039A0002E772093E80001C0B901FC0120E06115E9
:1039B000710579F1809119048823F1F18530F1F1D5
:1039C0008091E80083FD3CC08091E80082FD2EC01C
:1039D0008091E80080FFEBCF2091F3008091F2000E
:1039E00090E0922B6115710551F08830910538F403
:1039F00021912093F100615071090196F3CF21E0EC
:103A0000089709F020E08091E8008E778093E80025
:103A1000CECF2111CFCF0AC080911904882361F045
:103A2000853061F08091E80083FD0AC08091E80054
:103A300082FFF2CF80E0089582E0089583E0089548
:103A400081E0089520912004309121042617370742
:103A500048F06115710539F42091E8002E77209324
:103A6000E80001C0B901FC0120E06115710591F188
:103A700080911904882309F440C0853009F43FC0BF
:103A80008091E80083FD3DC08091E80082FD2FC059
:103A90008091E80080FFE9CF2091F3008091F2004F
:103AA00090E0922B6115710559F08830910540F432
:103AB00024912093F1003196615071090196F2CF63
:103AC00021E0089709F020E08091E8008E7780934C
:103AD000E800CBCF2111CCCF0AC0809119048823F4
:103AE00061F0853061F08091E80083FD0AC080912B
:103AF000E80082FFF2CF80E0089582E0089583E03D
:103B0000089581E008951F93CF93DF93CDB7DEB77B
:103B1000AA970FB6F894DEBF0FBECDBFEAE1F4E07E
:103B20008091F100819324E0E232F207C9F70E940C
:103B3000BD198091E80083FF2EC180911A049091F5
:103B40001B04492F50E04A30510508F024C1FA0106
:103B5000ED5BFE4F0C946C32803821F0823809F016
:103B60001AC108C08091160490911704992389F016
:103B700082600FC080911E048F70873008F00BC1E7
:103B80008093E9008091EB0085FB882780F91092F3
:103B9000E9009091E800977F9093E8008093F1000E
:103BA0001092F100D1C0282F2D7F09F0F4C0882396
:103BB00019F0823061F0EFC080911C04813009F06F
:103BC000EAC0933009F080E0809317042EC0809102
:103BD0001C0481112AC080911E048F702FEF280FC2
:103BE000263008F0D8C08093E9002091EB0020FF38
:103BF0001CC0933021F48091EB00806214C090913E
:103C0000EB0090619093EB0021E030E0A90102C04D
:103C1000440F551F8A95E2F74093EA001092EA009C
:103C20008091EB0088608093EB001092E900809116
:103C3000E800877F8093E8000E94251CACC08111BA
:103C4000AAC010911C041F778091E3008078812B1B
:103C50008093E3008091E800877F8093E8000E94D2
:103C6000251C8091E80080FFFCCF8091E3008068F4
:103C70008093E300111102C082E001C083E08093D1
:103C8000190489C08058823008F085C080911C04D6
:103C900090911D048C3D53E0950779F583E08A836C
:103CA0008AE289834FB7F894DE01139620E03EE064
:103CB00051E2E32FF0E050935700E49120FF03C05E
:103CC000E295EF703F5FEF708E2F90E0EA3010F0DA
:103CD000C79601C0C0968D939D932F5F243149F7FD
:103CE0004FBF8091E800877F8093E8006AE270E030
:103CF000CE0101960E94C41C16C060911E047091F2
:103D00001F04AE014F5F5F4F0E94841BBC01892BD3
:103D100009F441C09091E800977F9093E800898171
:103D20009A810E94221D8091E8008B778093E800A1
:103D300032C0803881F58091E800877F8093E80069
:103D4000809115048093F1008091E8008E7772CF06
:103D5000811121C080911C0490911D049927029724
:103D6000D4F48091E800877F8093E80080911C0460
:103D7000809315040E94251C80911504811106C0B2
:103D80008091E30087FD02C081E001C084E0809360
:103D900019040E94AE198091E80083FF0AC0809147
:103DA000E800877F8093E8008091EB008062809339
:103DB000EB00AA960FB6F894DEBF0FBECDBFDF9121
:103DC000CF911F9108950E94511F0E94591FE0EE4C
:103DD000F0E0808181608083E8EDF0E080818F7782
:103DE000808319BCA7EDB0E08C918E7F8C9380818D
:103DF0008F7E80831092180408950F931F93CF93A2
:103E0000DF930E94511F0E94591FC8EDD0E08881A6
:103E10008F77888388818068888388818F7D888375
:103E200019BC1092190410921504109217041092E4
:103E3000160400EE10E0F80180818B7F808388817A
:103E40008160888342E060E080E00E94F01BE1EE48
:103E5000F0E080818E7F8083E2EEF0E080818160FF
:103E60008083808188608083F80180818E7F808359
:103E7000888180618883DF91CF911F910F91089590
:103E8000E8EDF0E080818F7E8083E7EDF0E08081D7
:103E90008160808384E082BF81E0809318040C9469
:103EA000FD1EE8EDF0E080818E7F80831092E200BD
:103EB00008951092DA001092E10008951F920F9277
:103EC0000FB60F9211242F933F934F935F936F93ED
:103ED0007F938F939F93AF93BF93EF93FF938091C3
:103EE000E10082FF0BC08091E20082FF07C0809159
:103EF000E1008B7F8093E1000E942B208091DA000B
:103F000080FF1FC08091D80080FF1BC08091DA0025
:103F10008E7F8093DA008091D90080FF0DC080E110
:103F200089BD82E189BD09B400FEFDCF81E08093A7
:103F300019040E94A11905C019BC109219040E940D
:103F4000AA198091E10080FF19C08091E20080FFF2
:103F500015C08091E2008E7F8093E2008091E200A4
:103F600080618093E2008091D80080628093D800C5
:103F700019BC85E0809319040E94A51A8091E10084
:103F800084FF30C08091E20084FF2CC080E189BDB5
:103F900082E189BD09B400FEFDCF8091D8008F7DFC
:103FA0008093D8008091E1008F7E8093E100809122
:103FB000E2008F7E8093E2008091E2008160809336
:103FC000E20080911504882311F084E007C08091FD
:103FD000E30087FD02C081E001C083E08093190403
:103FE0000E94BA1A8091E10083FF24C08091E20010
:103FF00083FF20C08091E100877F8093E10082E011
:1040000080931904109215048091E1008E7F8093B3
:10401000E1008091E2008E7F8093E2008091E200D7
:1040200080618093E20042E060E080E00E94F01B4B
:104030000E94AD19FF91EF91BF91AF919F918F9128
:104040007F916F915F914F913F912F910F900FBE94
:104050000F901F9018950895CF938091190488238D
:10406000A1F0C091E900CF709091EC00892F817090
:1040700090FD80E8C82B1092E9008091E80083FD54
:104080000E94831DCF70C093E900CF910895909353
:104090001203809311030895E0911103F09112032C
:1040A000309721F00190F081E02D099480E008958F
:1040B000EF92FF920F931F93CF93DF93E091110341
:1040C000F09112033097B1F18C010280F381E02D61
:1040D00009958091070482FF2DC080FF04C08BEBFF
:1040E00097E00E94B804E80110E285EBE82E87E033
:1040F000F82E8091070480FF0BC088811F928F9358
:10410000FF92EF920E9451050F900F900F900F9029
:10411000115021961111EDCF8091070480FF0AC044
:1041200083EB97E0DF91CF911F910F91FF90EF907C
:104130000C94B804DF91CF911F910F91FF90EF90F5
:1041400008951F93CF93DF932091110330911203B1
:10415000232BB1F0EC0118810E9424319881892B26
:1041600088830E94A10C9881892B8883E091110398
:10417000F09112030480F581E02DCE01099518839A
:10418000DF91CF911F910895CF93DF9320910F037B
:10419000309110032817390709F190931003809389
:1041A0000F03E0911103F09112033097B9F0EC0185
:1041B0000680F781E02D09958091070482FF0EC0EB
:1041C00080FF0CC0DF93CF9385EA97E09F938F9396
:1041D0000E9451050F900F900F900F90DF91CF919B
:1041E0000895CF93DF9320910D0330910E0328178C
:1041F000390709F190930E0380930D03E0911103A9
:10420000F09112033097B9F0EC010084F185E02DB4
:1042100009958091070482FF0EC080FF0CC0DF93D8
:10422000CF9385E997E09F938F930E9451050F905C
:104230000F900F900F90DF91CF9108950C94DF2194
:104240000E94FE2D0C94780C8F929F92AF92BF9299
:10425000CF92DF92EF92FF920F931F93CF93DF9352
:1042600000D000D01F92CDB7DEB70E94781704E1CE
:1042700013E0F12C8F2D0E947F0C4C01F801A080DF
:10428000B180A826B926A114B10439F4F3940E5FC5
:104290001F4FF8E0FF12EECF39C08091070481FD77
:1042A0000E94F321E12CCC24C394D12CC5018C2194
:1042B0009D21892B21F1E982FA8221E0C4018C2120
:1042C0009D21892B09F420E02B830E94072E816019
:1042D000782F9D838C8349815A816B818D810E94C7
:1042E000292249815A816B817C818D810E949E2D7A
:1042F000F801808191818C259D2591838083E394B1
:10430000CC0CDD1CF0E1EF12D1CFC0CF8FEF898351
:104310008A831B820E94072E8160782F9D838C8365
:1043200049815A816B818D810E9429220E949D2D95
:104330000E9473300E944C2090911303891759F109
:104340000E944C20809313039091070492FF0EC0AB
:1043500090FF0CC01F928F9386EC97E09F938F93F2
:104360000E9451050F900F900F900F9080911303B2
:104370000F900F900F900F900F90DF91CF911F91A2
:104380000F91FF90EF90DF90CF90BF90AF909F90F4
:104390008F900C94AF2D0F900F900F900F900F9067
:1043A000DF91CF911F910F91FF90EF90DF90CF9011
:1043B000BF90AF909F908F9008950C94B70C089584
:1043C000CF93C62F0E947F0C21E030E002C0220F65
:1043D000331FCA95E2F72823392381E0232B09F400
:1043E00080E0CF910895EF92FF920F931F93CF93A8
:1043F000DF938DED97E00E94B804C0E0D0E080E24A
:10440000E82E81E0F82E01ED17E08C2F0E947F0C42
:104410000E94892DFF92EF929F938F93DF93CF930A
:104420001F930F930E94510521968DB79EB7089652
:104430000FB6F8949EBF0FBE8DBFC830D10529F7C7
:10444000DF91CF911F910F91FF90EF900895089504
:104450000895CF93DF93CDB7DEB72B970FB6F894BF
:10446000DEBF0FBECDBF942F4F83252F588769879E
:104470007A878B874A855B85452B31F02F3F31F456
:1044800081E09F3F19F403C081E001C080E080FD1E
:1044900007C04F81588569857A858B850E949E2D3E
:1044A000DE01119686E0FD0111928A95E9F785E01B
:1044B000FE01379601900D928A95E1F749815A8164
:1044C0006B817C818D819E810E948F292B960FB6F6
:1044D000F894DEBF0FBECDBFDF91CF910895882342
:1044E00009F4BBC09CEF980F913A18F40E946D2C10
:1044F0000DC090E2980F983058F4877091E001C099
:10450000990F8A95EAF7892F0E94122D0C944C2D51
:104510009BE5980F933070F4853A29F0863A31F094
:1045200083E890E005C081E890E002C082E890E076
:104530000C94C42098E5980F973108F08EC0883A03
:1045400009F445C0893A09F445C08A3A09F445C0DE
:104550008B3A09F445C08C3A09F445C08D3A09F408
:1045600045C08E3A09F445C08F3A09F445C0813BF5
:1045700009F445C0803B09F445C0823B09F445C0BD
:10458000833B09F445C0843B09F445C0853B09F4ED
:1045900045C0863B09F445C0873B09F445C0883BCC
:1045A00009F445C0893B09F445C08A3B09F445C07C
:1045B0008B3B09F445C08C3B09F445C08D3B09F4A5
:1045C00045C08E3B09F445C080E090E044C082EED7
:1045D00090E041C089EE90E03EC08AEE90E03BC0A2
:1045E00085EB90E038C086EB90E035C083EB90E03F
:1045F00032C084EB90E02FC087EB90E02CC08CECB5
:1046000090E029C08DEC90E026C083E891E023C0C3
:104610008AE891E020C082E991E01DC084E991E040
:104620001AC081E292E017C083E292E014C084E2F3
:1046300092E011C085E292E00EC086E292E00BC0EB
:1046400087E292E008C08AE292E005C08FE690E03F
:1046500002C080E790E00C94F1200895882329F1AE
:104660009CEF980F913A18F40E94BD2C0DC090E277
:10467000980F983058F4877091E001C0990F8A958F
:10468000EAF7892F0E94182D0C944C2D9BE5980F6A
:10469000933020F480E090E00C94C420885A873155
:1046A00020F480E090E00C94F1200895882321F01C
:1046B0000E94122D0C944C2D0895882321F00E9405
:1046C000182D0C944C2D08950E94322D0E94012D1E
:1046D0000E944C2D0E9418310E94E62F80E090E04D
:1046E0000E94C42080E090E00C94F1200E94222DD2
:1046F0000C946423CF92DF92EF92FF920F931F935B
:10470000CF93DF9300D000D01F92CDB7DEB76C01FE
:104710000E94B12D811118C385E0F601DE011196CA
:1047200001900D928A95E1F7F60140815181238134
:1047300034812115310531F05F3F31F481E04F3F85
:1047400019F403C081E001C080E080FDFDC2F601E4
:10475000F280E580E2948FE0E82249835A83FB826D
:10476000722F3D832C836F2D8D810E94E92B8C014C
:104770000E94E82B0E94E22AE12FE295EF708E2F33
:1047800090E0FC01E35BFE4F0C946C32812F807F44
:104790001F70882311F01295107FFF20B9F01123AC
:1047A00029F0812F0E94252D0E944C2D802F0F90E3
:1047B0000F900F900F900F90DF91CF911F910F915D
:1047C000FF90EF90DF90CF900C946F22802F0E948B
:1047D0002E23112309F4B8C2812F0E942B2D0F9094
:1047E0000F900F900F900F90DF91CF911F910F912D
:1047F000FF90EF90DF90CF900C944C2D812F807F15
:104800001F70803211F01295107F002319F00130D3
:1048100009F12BC0FF20A9F0EE2059F1F1E0812F22
:10482000EF1228C00F900F900F900F900F90DF9114
:10483000CF911F910F91FF90EF90DF90CF900C944C
:10484000352DEE2021F021E0E21609F47DC20E9410
:10485000382D4DC0FF20E9F085E08E1508F474C2B4
:104860000E940F2D812329F042C0FF20F1F1E110B9
:1048700015C0812F0F900F900F900F900F90DF9128
:10488000CF911F910F91FF90EF90DF90CF900C94FC
:10489000562394E09E1508F457C229C0F60185817D
:1048A00080FF13C08F708583E4CF003F09F489C176
:1048B00008F055C180E4800F803208F459C1FF2010
:1048C00009F4EAC1EE2009F49AC1802F0E946F22F8
:1048D000093309F0DAC1FFEF21EE84E0F150204006
:1048E0008040E1F700C000002FC2E110D7C1812F46
:1048F00059C1812F86958695837019F08130B9F062
:1049000023C2FF2019F0C801937002C080E090E03C
:104910000F900F900F900F900F90DF91CF911F91FC
:104920000F91FF90EF90DF90CF900C94C420FF2068
:1049300019F0C801937002C080E090E00F900F90D2
:104940000F900F900F90DF91CF911F910F91FF90DB
:10495000EF90DF90CF900C94F120802FFF2019F082
:104960000E94F92E02C00E94612F0F900F900F90AD
:104970000F900F90DF91CF911F910F91FF90EF90CB
:10498000DF90CF900C94E62F812F837009F070C0D8
:10499000F110DAC1202F229526952770220F220FC1
:1049A000602F6F70862F90E0A0E0B0E06C017D0179
:1049B000022E04C0CC0CDD1CEE1CFF1C0A94D2F7A6
:1049C00004FF12C08FE090E0A0E0B0E004C0880FC8
:1049D000991FAA1FBB1F2A95D2F7BC01CD01609574
:1049E00070958095909503C060E070E0CB011695BE
:1049F000169513701230B1F040F56C297D298E297F
:104A00009F29113031F10F900F900F900F900F9060
:104A1000DF91CF911F910F91FF90EF90DF90CF909A
:104A20000C94FD2A6C297D298E299F290F900F90C7
:104A30000F900F900F90DF91CF911F910F91FF90EA
:104A4000EF90DF90CF900C94172B0E94FD2AC701A6
:104A5000B6010F900F900F900F900F90DF91CF91B4
:104A60001F910F91FF90EF90DF90CF900C94E32A6D
:104A7000FF2019F0812F817001C08695882309F4E9
:104A800063C1202F229526952770220F220F602FB9
:104A90006F70862F90E0A0E0B0E06C017D01022EE7
:104AA00004C0CC0CDD1CEE1CFF1C0A94D2F704FFE2
:104AB00012C08FE090E0A0E0B0E004C0880F991F22
:104AC000AA1FBB1F2A95D2F7BC01CD016095709536
:104AD0008095909503C060E070E0CB011695169527
:104AE00013701230B1F040F56C297D298E299F2971
:104AF000113031F10F900F900F900F900F90DF91C8
:104B0000CF911F910F91FF90EF90DF90CF900C9479
:104B1000C42B6C297D298E299F290F900F900F900F
:104B20000F900F90DF91CF911F910F91FF90EF9019
:104B3000DF90CF900C94D62B0E94C42BC701B601F6
:104B40000F900F900F900F900F90DF91CF911F91CA
:104B50000F91FF90EF90DF90CF900C94B22B023F1B
:104B600009F45EC008F449C0033F09F46CC0A7CE45
:104B7000902F9071E92E812F8F71FF2051F00E94AC
:104B80004B2B802FEE2019F08295807F73CE8F7093
:104B900071CE0E946C2B802FEE2019F08295807FC1
:104BA00001C08F700F900F900F900F900F90DF91BA
:104BB000CF911F910F91FF90EF90DF90CF900C94C9
:104BC0005D23FF20A9F0E4E0EE1508F4BDC0812FBD
:104BD0008F710F900F900F900F900F90DF91CF91EA
:104BE0001F910F91FF90EF90DF90CF900C94912B3D
:104BF000F5E0FE1508F4A8C0EACFFF2099F0812F58
:104C00008F710F900F900F900F900F90DF91CF91B9
:104C10001F910F91FF90EF90DF90CF900C944B2B52
:104C2000FF2069F3812F8F710F900F900F900F90DD
:104C30000F90DF91CF911F910F91FF90EF90DF9038
:104C4000CF900C946C2BFF2089F0812F8F710F90E7
:104C50000F900F900F900F90DF91CF911F910F91B8
:104C6000FF90EF90DF90CF900C94362B0F900F9029
:104C70000F900F900F90DF91CF911F910F91FF90A8
:104C8000EF90DF90CF900C94312B033509F423CEB5
:104C9000073409F059C01FCEEE2021F2802F0F906B
:104CA0000F900F900F900F90DF91CF911F910F9168
:104CB000FF90EF90DF90CF900C942E23412F4F70F8
:104CC000602FC6010E94732E0F900F900F900F90CF
:104CD0000F90DF91CF911F910F91FF90EF90DF9098
:104CE000CF900C943D2A01112FC0FF2069F10E9442
:104CF00076232FEF80E792E0215080409040E1F74B
:104D000000C000000F900F900F900F900F90DF9158
:104D1000CF911F910F91FF90EF90DF90CF900C9467
:104D2000542E412F4F70602FC6010F900F900F909F
:104D30000F900F90DF91CF911F910F91FF90EF9007
:104D4000DF90CF900C94762E0F900F900F900F90D5
:104D50000F90DF91CF911F910F91FF90EF90DF9017
:104D6000CF9008951F93CF93DF9300D000D01F9270
:104D7000CDB7DEB7942F4983252F5A836B837C836D
:104D80008D834C815D81452B31F02F3F31F481E0E3
:104D90009F3F19F403C081E001C080E0182F11701B
:104DA00080FD24C049815A816B817C818D810E9464
:104DB000E92B292F22952F702C3030F42A3048F41B
:104DC0002250223068F013C02C3061F02F3051F0A7
:104DD0000EC0803C28F0803E50F0815F833038F078
:104DE00011E005C093FB112710F901C010E0812FDD
:104DF0000F900F900F900F900F90DF91CF911F9118
:104E00000895CF93DF9300D000D01F92CDB7DEB7C7
:104E10000F900F900F900F900F90DF91CF9108950A
:104E2000CF93DF9300D000D000D0CDB7DEB7269669
:104E30000FB6F894DEBF0FBECDBFDF91CF910895BE
:104E40001F93CF93DF93C091240316E08091250335
:104E5000C81799F0D0E01C9FF0011D9FF00D1124A0
:104E6000EA5DFC4F4081518162817381848195812B
:104E70000E9410272196C770E9CFDF91CF911F9133
:104E800008954091560350915703609158037091D3
:104E9000590380915A0390915B030C9410270F9350
:104EA0001F93CF93DF9380915B0382958F7009F0FE
:104EB0005DC080915803882309F458C08091240371
:104EC000109125036091560370915703C0915903C7
:104ED000D0915A0391E06F3F09F090E0292F06E04E
:104EE000811709F443C0209721F07F3F21F030E083
:104EF00003C031E001C0322F90E030FD34C0089F84
:104F0000F001099FF00D1124DF01AA5DBC4F11963D
:104F10003C911197371327C03C91361324C0129649
:104F20003C91129731111FC013964D915C911497CB
:104F30004C1B5D0B483C5105B0F480915B038F70B6
:104F4000806180935B03E55DFC4F80818F708061A1
:104F5000808386E593E00E947A23DF91CF911F91B1
:104F60000F910C94202701968770BACFDF91CF91D3
:104F70001F910F9108959F92AF92BF92CF92DF92AF
:104F8000EF92FF920F931F93CF93DF93CDB7DEB7CE
:104F900061970FB6F894DEBF0FBECDBF8C0185E0E0
:104FA000F801DE011D9601900D928A95E1F7F80156
:104FB00040815181F280C380D480909156036091EA
:104FC00057032091590330915A032115310531F0CF
:104FD0006F3F31F481E09F3F19F403C081E001C0CD
:104FE00080E0F82FF1709F2E80FD52C186E5A82E3B
:104FF00083E0B82EE0905803F601E21BF30BEE209D
:1050000009F4E8C080915B03E83CF10508F0A4C016
:10501000282F207F09F053C0561313C0491311C025
:10502000EF2CF1100EC08F70806180935B030E94A3
:105030004127C5010E947A2380915B03F801858393
:105040005BC1C114D10431F05F3F31F481E04F3FC7
:1050500019F403C081E001C080E080FD03C081E05D
:105060008F2502C080E090E0F82FF170EF2E80FFD6
:105070001CC0809124032091250336E0821709F497
:1050800018C190E0389FF001399FF00D1124EA5DBE
:10509000FC4F6181561306C06081461303C06281D4
:1050A000F61203C001968770E9CFEF2CFF2009F4B8
:1050B00023C180915B03816080935B0362C05613C0
:1050C00006C0491304C0F11002C0F801A7C04D8703
:1050D0005E87FF867C2DD98AC88A6F2D89890E94B8
:1050E000B226882399F1FF2089F120915B03822F5A
:1050F00082958F7090E0029774F0809156039091A2
:10510000570398878F831986DB86CA862C87CE0142
:1051100007960E947A2386E0F801A6E5B3E00190A5
:105120000D928A95E1F70E944F270E94412711C0F6
:10513000561749F14D875E87FF867C2DD98AC88A2C
:105140006F2D89890E94B22681112CC0C8010E944E
:105150007A23EE24E394D0C0282F207F49F77C2DBA
:10516000D98AC88A6F2D89890E94012786E593E034
:105170000E947A2386E0F50111928A95E9F70E9450
:105180004127E12CB9C04913D5CFF110D3CFF80195
:105190008583C8010E947A2386E0F50111928A95E1
:1051A000E9F7AAC0FF2091F220915B03822F82953C
:1051B0008F7090E002970CF4AECF809156039091DF
:1051C00057039A8389831B82DD82CC822E83CE0192
:1051D00001969FCFE83CF10508F04BC0EF2CFF2073
:1051E00009F4B4CF561330C049132EC020915B038D
:1051F00020FD21C0822F82958F70482F50E04115ED
:105200005105C9F0F80125834F30510541F08F5FFA
:10521000982F9295907F822F8F70892B8583C8015C
:105220000E947A2386E0F801A6E5B3E001900D9292
:105230008A95E1F72AC086E0F801A6E5B3E001907F
:105240000D928A95E1F758C04D875E87FF867C2DC9
:10525000D98AC88A6F2D89890E94B22681115BCFB5
:1052600080915B03816080935B03C8010E947A2375
:1052700043C07C2DD98AC88A6F2D89890E94012755
:1052800086E0F50111928A95E9F70E94412734C022
:10529000FF2009F45BCF4D875E87FF867C2DD98A7E
:1052A000C88A6F2D89890E94B226882309F44ECFBF
:1052B00032CF7C2DD98AC88A6F2D89890E94E92B2B
:1052C000292F22952F70223028F49F7039F08111F8
:1052D00005C00BC0243028F49F7049F4805E8830EC
:1052E00020F0C8010E947A239E2CE92C05C0F80109
:1052F0009581907F99F7F9CF8E2D61960FB6F8942E
:10530000DEBF0FBECDBFDF91CF911F910F91FF90F8
:10531000EF90DF90CF90BF90AF909F9008951F9334
:10532000CF93DF93CDB7DEB72C970FB6F894DEBFDF
:105330000FBECDBF4F83588769877A878B879C873D
:10534000CE0107960E94BB278823D1F09F818885D4
:105350002A853B85232B31F08F3F31F481E09F3F3D
:1053600019F403C081E001C080E080FD47C04F8197
:10537000588569857A858B859C850E9410273EC05B
:1053800086E0FE013796DE01119601900D928A9516
:10539000E1F7FF81E8856A857B856115710531F04C
:1053A000EF3F31F481E0FF3F19F403C081E001C019
:1053B00080E080FD23C02091250330E0C9010196E3
:1053C000877099274091240350E084179507F1F1E5
:1053D000F983EA837D836C8396E0929FD001939F4B
:1053E000B00D1124AA5DBC4FFE01319601900D92C3
:1053F0009A95E1F7809325030E94202716E080917B
:10540000240390912503891771F1189FC00111247D
:105410008A5D9C4F0E94BB27882329F1E0912403D9
:105420001E9FF0011124EA5DFC4F40815181628191
:105430007381848195810E9410278091240390E0DC
:1054400001968770992780932403D9CF0E947623F1
:105450001092250310922403E6E5F3E086E0DF01D5
:105460001D928A95E9F72C960FB6F894DEBF0FBE11
:10547000CDBFDF91CF911F910895DF92EF92FF9200
:105480000F931F93CF93DF93FC01892B09F488C0FE
:10549000E12CF12CDD24D394EF0121968491853702
:1054A00009F460C058F4843708F04EC0843008F026
:1054B00068C08130D1F0823071F172C0883709F450
:1054C0005BC050F4863709F453C0873709F068C0D1
:1054D0008E2D0E941F2D52C09CE7980F903708F028
:1054E0005FC08F770E942E234EC08F010E5F1F4F2B
:1054F000FE01849190E2980F983050F48770FD2D52
:1055000001C0FF0F8A95EAF78F2F0E94252D15C045
:105510000E946F2214C08F010E5F1F4FFE01849105
:1055200090E2980F983068F48770FD2D01C0FF0F4E
:105530008A95EAF78F2F0E942B2D0E944C2DE801AF
:1055400022C00E942E23FBCFCF010296FE01C49100
:10555000CC2361F0EFE9FFE03197F1F700C00000E4
:10556000C150F6CFCF010296FE01F490EC010BC0C2
:105570000E940F2DE82E07C00E94222D0E944C2D64
:1055800002C00E946F228F2D882341F0EFE9FFE0D7
:105590003197F1F700C000008150F6CFFE017CCFBB
:1055A000DF91CF911F910F91FF90EF90DF900895C1
:1055B0006093DC037093DD038093DE039093DF033D
:1055C0000C94AE2D08950F931F930091E00310915A
:1055D000E1032091E2033091E303602B712B822BD6
:1055E000932B6093E0037093E1038093E203909325
:1055F000E3031F910F910C94AD2D0F931F93009116
:10560000E0031091E1032091E2033091E303602372
:105610007123822393236093E0037093E1038093CB
:10562000E2039093E3031F910F910C94AD2D0F9320
:105630001F930091E0031091E1032091E203309168
:10564000E30360277127822793276093E003709319
:10565000E1038093E2039093E3031F910F910C9475
:10566000AD2D60E070E0CB010C94D82A0F931F930E
:1056700041E050E060E070E08A019B0104C0000F4F
:10568000111F221F331F8A95D2F7C901B8011F913C
:105690000F910C94D82A0F931F9341E050E060E0E3
:1056A00070E004C0440F551F661F771F8A95D2F71C
:1056B0008091DC039091DD03A091DE03B091DF03C4
:1056C0008A019B01082B192B2A2B3B2BC901B801FE
:1056D0001F910F910C94D82A0F931F9341E050E033
:1056E00060E070E004C0440F551F661F771F8A9565
:1056F000D2F740955095609570958091DC0390911C
:10570000DD03A091DE03B091DF038A019B01082332
:1057100019232A233B23C901B8011F910F910C942F
:10572000D82A0F931F9341E050E060E070E004C07E
:10573000440F551F661F771F8A95D2F78091DC03AF
:105740009091DD03A091DE03B091DF038A019B01FC
:10575000082719272A273B27C901B8011F910F9154
:105760000C94D82A0F931F930091DC031091DD0352
:105770002091DE033091DF03602B712B822B932B62
:105780001F910F910C94D82A0F931F930091DC0363
:105790001091DD032091DE033091DF03602371233C
:1057A000822393231F910F910C94D82A0F931F9358
:1057B0000091DC031091DD032091DE033091DF03C3
:1057C00060277127822793271F910F910C94D82A65
:1057D00008958F929F92AF92BF92DF92EF92FF92C5
:1057E0000F931F93CF93DF9300D000D01F92CDB7BC
:1057F000DEB76B837C838D838A018C819D81892BAD
:1058000031F01F3F31F481E04F3F19F403C081E0D4
:1058100001C080E080FF03C080E090E04DC08B813C
:105820008823D1F18090DC039090DD03A090DE030B
:10583000B090DF038091E0039091E103A091E20337
:10584000B091E303882A992AAA2ABB2A8FE1E82E7D
:10585000F12CD501C4010E2C04C0B695A7959795DF
:1058600087950A94D2F780FD06C081E0E81AF10816
:1058700080F7D12C07C0DE2CB8018E2D0E948A0C37
:10588000019799F380E1189FF0011124E45AFC4F2D
:10589000E00FF11DD08209C080E1189FF0011124B2
:1058A000E45AFC4FE00FF11DD08009831A8369810F
:1058B0007A818D2D0E948A0C0F900F900F900F907F
:1058C0000F90DF91CF911F910F91FF90EF90DF909C
:1058D000BF90AF909F908F90089590911101992360
:1058E00079F190911201992359F1982F96959695F7
:1058F00096959F31A1F0E0911301F0911401E90F09
:10590000F11D877021E030E0A90102C0440F551F4E
:105910008A95E2F7CA019181892B8183089590913C
:10592000070490FF29C01F928F9380E198E09F9316
:105930008F930E9451050F900F900F900F90089534
:105940002091130130911401F90132969FEF40E04C
:105950005191851789F09F3F19F4511101C0942F7F
:105960004F5F4E31A9F79F3F39F0F901E90FF11D63
:1059700097FDFA95828308950895909111019923D6
:1059800081F190911201992361F1982F9695969546
:1059900096959F31A9F0E0911301F0911401E90F60
:1059A000F11D877021E030E0A90102C0440F551FAE
:1059B0008A95E2F7CA0180959181892381830895B0
:1059C0009091070490FF1CC01F928F9382EF97E085
:1059D0009F938F930E9451050F900F900F900F90FF
:1059E0000895E0911301F09114019F01225E3F4F51
:1059F0009281891301C012823196E217F307C1F731
:105A0000089581E090E0E0911301F0911401E80F16
:105A1000F91F1082019680329105A9F708958091AF
:105A20000604089590910604892B80930604089536
:105A300080959091060489238093060408958093AD
:105A40000604089510920604089590910504892B88
:105A5000809305040895809590910504892380938F
:105A6000050408951092050408958093E4030895B1
:105A70001092E40308958091130190911401FC01A8
:105A800031969C01205E3F4F80E0919191118F5F94
:105A9000E217F307D1F70895E0911301F091140193
:105AA000809106048083E0911301F09114019081AC
:105AB00080910504892B80838091E403882361F021
:105AC000E0911301F09114019081892B80830E9451
:105AD0003B2D81111092E4038091130190911401E8
:105AE0000C94582090937F0180937E0108958295B5
:105AF000982F937344E0949F900111248C7C869599
:105B00008695282B822F8575880F2A7A2695822BD9
:105B10000895CF93DF93D92F0E94772DC82F8D2F13
:105B20000E94772D2C2F30E0322F2227A901482BFD
:105B3000CA01DF91CF91089508950895CF93DF931F
:105B400000D000D01F92CDB7DEB70F900F900F900E
:105B50000F900F90DF91CF910895089508950C94C0
:105B6000DD2180E0089583B7817F8C6083BF83B798
:105B7000816083BF7894889583B78E7F83BF0895B3
:105B8000CF930E9427220E9478170E942822C0E00B
:105B90008C2F0E947F0C892B29F4CF5FC830C1F76E
:105BA00080E001C081E0CF9108950E94880C0C94A0
:105BB00076231F920F920FB60F9211248F939F930B
:105BC000AF93BF938091080490910904A0910A04B7
:105BD000B0910B044196A11DB11D809308049093D0
:105BE0000904A0930A04B0930B04BF91AF919F9155
:105BF0008F910F900FBE0F901F90189582E084BD7B
:105C000093E095BD9AEF97BD80936E0008952FB7EE
:105C1000F8948091080490910904A0910A04B0912D
:105C20000B042FBF08952FB7F8946091080470916A
:105C3000090480910A0490910B042FBF08959C01E0
:105C40004FB7F8948091080490910904A0910A0438
:105C5000B0910B044FBF821B930B089578941F9251
:105C60000F920FB60F9211248F939F93AF93BF9310
:105C70008091080490910904A0910A04B0910B044A
:105C80000196A11DB11D8093080490930904A0936F
:105C90000A04B0930B04BF91AF919F918F910F9025
:105CA0000FBE0F901F9018950E94E31EF89487E78F
:105CB00097E7909301088093000887E090EBDC0160
:105CC0008093220490932304A0932404B09325048A
:105CD0009CE088E10FB6F894A895809360000FBE11
:105CE00090936000FFCF80E090E008950895809148
:105CF0000E0480FF0BC06091180185E0689FB00121
:105D0000112475956795759567952BC081FF09C01E
:105D10006091180185E0689FB00111247595679521
:105D200020C082FF07C06091180185E0689FB00124
:105D3000112417C090910F049923D1F0609117019D
:105D4000961788F72091180185E0289F900111246B
:105D5000929FA001939F500D112470E0CA010E94F0
:105D600058326038710540F46115710519F406C0A8
:105D700065E070E0862F08958FE7089581E008952B
:105D800080910E0480FF08C06091160170E0759547
:105D900067957595679521C081FF06C060911601D2
:105DA00070E07595679519C082FF04C06091160177
:105DB00070E010C090910F04992399F06091150143
:105DC0009617A0F780911601899FC001112470E0F9
:105DD0000E9458326038710540F46115710519F45C
:105DE00006C061E070E0862F08958FE7089581E096
:105DF0000895803F21F40E94772E819504C0813F51
:105E000029F40E94772E809312040895823F21F492
:105E10000E94772E819504C0833F29F40E94772E3B
:105E2000809311040895893F19F40E94C02E05C083
:105E30008A3F31F40E94C02E819580931304089507
:105E40008B3F21F40E94C02E819504C08C3F29F421
:105E50000E94C02E809314040895843F21F4809101
:105E60001004816017C0853F21F480911004826086
:105E700011C0863F21F48091100484600BC0873FDD
:105E800021F480911004886005C0883F31F480912E
:105E9000100480618093100408958D3F21F4809157
:105EA0000E0481600BC08E3F21F480910E0482604D
:105EB00005C08F3F29F480910E04846080930E0406
:105EC0000895803F39F48091120487FF6CC01092CE
:105ED000120469C0813F29F4809112041816BCF3A2
:105EE00062C090911104823F29F497FF5CC0109228
:105EF000110459C0833F19F41916CCF354C0893FDB
:105F000041F48091130418160CF04DC01092130444
:105F10004AC08A3F29F48091130487FF44C0F6CF1A
:105F20008B3F39F48091140487FF3DC01092140414
:105F30003AC08C3F29F4809114041816BCF333C086
:105F4000843F21F4809110048E7F17C0853F21F497
:105F5000809110048D7F11C0863F21F48091100440
:105F60008B7F0BC0873F21F480911004877F05C091
:105F7000883F31F4809110048F7E8093100413C009
:105F80008D3F21F480910E048E7F0BC08E3F21F453
:105F900080910E048D7F05C08F3F29F480910E04FF
:105FA0008B7F80930E048091110481110EC080912B
:105FB000120481110AC080911304811106C08091DE
:105FC0001404811102C010920F04089580910704F7
:105FD00083FF7EC085E598E00E94B804809110049C
:105FE0001F928F9380E598E09F938F930E945105B5
:105FF0008EE498E00E94B80480911104282F082EA6
:10600000000C330B3F938F938BE498E09F938F9317
:106010000E94510589E498E00E94B804809112041E
:10602000282F082E000C330B3F938F9386E498E0C3
:106030009F938F930E94510584E498E00E94B804D6
:1060400080911304282F082E000C330B3F938F935D
:1060500081E498E09F938F930E9451058FE398E02D
:106060000E94B80480911404282F082E000C330BD2
:106070003F938F938CE398E09F938F930E945105F9
:1060800089E398E00E94B80480910F041F928F93D7
:1060900086E398E09F938F930E94510584E398E0F4
:1060A0000E94B80480910E041F928F9381E398E0C0
:1060B0009F938F930E9451058EE298E00E94B8044E
:1060C0008DB79EB74C960FB6F8949EBF0FBE8DBF8E
:1060D00080E194E00E94A1200E94072E90930D047D
:1060E00080930C0408951F93CF93DF9380910C0449
:1060F00090910D040E941F2EAC0190910F049923E2
:1061000021F02091190130E006C020911A018AE0A7
:10611000289F900111244217530708F485C08091ED
:106120001104C0911204D091130410911404811130
:1061300007C0C11175C0D11173C0111171C074C0F5
:106140009F3F19F09F5F90930F04181624F40E944C
:10615000772E809311048091110487FF05C00E945F
:10616000772E8195809311041C1624F40E94772EBB
:10617000809312048091120487FF05C00E94772E3D
:1061800081958093120460911104662331F1C091CE
:106190001204CC2311F1062E000C770B880B990BFF
:1061A0000E945F3123E333E343E35FE30E94C331A3
:1061B0000E942731609311046C2FCC0F770B880B52
:1061C000990B0E945F3123E333E343E35FE30E94D3
:1061D000C3310E942731609312041D1624F40E94DB
:1061E000C02E809313048091130487FF05C00E9482
:1061F000C02E819580931304111624F40E94C02EA2
:10620000809314048091140487FF05C00E94C02E5F
:10621000819580931404DF91CF911F910C94E62F08
:106220009F3F09F08FCFA0CFDF91CF911F910895AD
:10623000E0E1F4E085E0DF011D928A95E9F7109234
:106240000F0410920E0408958091100408950E9486
:106250002E316894B1110C94BD3108950E94A23181
:1062600088F09F5798F0B92F9927B751B0F0E1F017
:10627000660F771F881F991F1AF0BA95C9F714C0C7
:10628000B13091F00E94BC31B1E008950C94BC3162
:10629000672F782F8827B85F39F0B93FCCF3869500
:1062A00077956795B395D9F73EF49095809570955D
:1062B00061957F4F8F4F9F4F0895E89409C097FBDA
:1062C0003EF490958095709561957F4F8F4F9F4FCD
:1062D0009923A9F0F92F96E9BB279395F695879511
:1062E00077956795B795F111F8CFFAF4BB0F11F4D4
:1062F00060FF1BC06F5F7F4F8F4F9F4F16C088237B
:1063000011F096E911C0772321F09EE8872F762FB0
:1063100005C0662371F096E8862F70E060E02AF0F1
:106320009A95660F771F881FDAF7880F96958795DD
:1063300097F9089557FD9058440F551F59F05F3F46
:1063400071F04795880F97FB991F61F09F3F79F097
:1063500087950895121613061406551FF2CF469519
:10636000F1DF08C0161617061806991FF1CF86959B
:106370007105610508940895E894BB27662777277F
:10638000CB0197F908950E94D6310C9447320E94B0
:10639000393238F00E94403220F0952311F00C94ED
:1063A00030320C94363211240C94BD310E949A3153
:1063B00070F3959FC1F3950F50E0551F629FF00158
:1063C000729FBB27F00DB11D639FAA27F00DB11D71
:1063D000AA1F649F6627B00DA11D661F829F2227FA
:1063E000B00DA11D621F739FB00DA11D621F839F81
:1063F000A00D611D221F749F3327A00D611D231F57
:10640000849F600D211D822F762F6A2F11249F57A4
:1064100050409AF0F1F088234AF0EE0FFF1FBB1FA7
:10642000661F771F881F91505040A9F79E3F510566
:1064300080F00C9430320C94BD315F3FE4F3983E11
:10644000D4F3869577956795B795F795E7959F5F10
:10645000C1F7FE2B880F911D9695879597F90895A2
:1064600097F99F6780E870E060E008959FEF80EC07
:10647000089500240A9416161706180609060895AA
:1064800000240A9412161306140605060895092E10
:106490000394000C11F4882352F0BB0F40F4BF2B7F
:1064A00011F460FF04C06F5F7F4F8F4F9F4F0895BF
:1064B00097FB072E16F4009407D077FD09D00E94B1
:1064C000723207FC05D03EF4909581959F4F089558
:1064D000709561957F4F0895EE0FFF1F0590F49121
:1064E000E02D0994AA1BBB1B51E107C0AA1FBB1FCB
:1064F000A617B70710F0A61BB70B881F991F5A9550
:10650000A9F780959095BC01CD010895F894FFCF2F
:1065100005EB010000FFA41746181718DB17A71793
:10652000010101E5032808140A321E5F5A31353093
:10653000005F3F3F3F3F005F41543834004154000B
:106540005854005445524D494E414C004E4F4E4513
:10655000004D4F55534500494E54454C4C49004C55
:106560004F474954454348004558504C4F524552B7
:106570000044454641554C5400397F225C07DD06F6
:0E658000BB06670680069906000800040002AC
:106800008800EA44E944E244040005000600070069
:10681000080009000A000B000C000D000E000F001C
:1068200010001100120013001400150016001700CC
:10683000180019001A001B001C001D001E001F007C
:10684000200021002200230024002500260027002C
:10685000280029002A002B002C002D002E002F00DC
:10686000300031003200330034003500360037008C
:10687000380039003A003B003C003D003E003F003C
:1068800040004100420043004400450046004700EC
:10689000480049004A004B004C004D004E004F009C
:1068A000500051005200530054005500560057004C
:1068B000580059005A005B005C005D005E005F00FC
:1068C0006000610062006300640065A185006700EC
:1068D000680069006A006B006C006D006E006F005C
:1068E0007000710072007300890087008A008B00BD
:1068F000E000E100E200E300E400E500E600E7007C
:106900000100010001000100EA4401000100E2442D
:106910000100010001000100460001004A004B0097
:10692000010001004700480001000100E9440100A6
:106930000100010001000100010001003A003B00DC
:106940003C003D003E003F0040004100420043004B
:10695000010035004C0039000100440045005200A0
:1069600049000100010050004F0029004D004E0079
:1069700051000100010001000100010001000100BF
:1069800001000100010001000100010001000100FF
:1069900001000100010001000100010001004D00A3
:1069A0004A004E004B0001000100010001000100FF
:1069B00001000100010001000100010001000100CF
:1069C00001000100010001000100010001000100BF
:1069D00001000100010001000100010001000100AF
:1069E0000100010001000100490001000100010057
:1069F000010001000100010001000100010001008F
:00000001FF
